:1000000012C02CC02BC02AC029C028C027C026C0BF
:1000100025C024C023C022C021C020C01FC01EC0D4
:100020001DC0E9C01BC011241FBECFE5D4E0DEBF58
:10003000CDBF10E0A0E6B0E0ECE2F3E002C0059036
:100040000D92AE36B107D9F710E0AEE6B0E001C0D0
:100050001D92A037B107E1F702D066C1D1CFCF938F
:1000600014BE88E10FB6F89481BD11BC0FBE86E0C6
:1000700087BB8CE084BB11BA82E411D12ED03DD075
:1000800078942DE088E190E00FB6F894A89581BDB2
:100090000FBE21BD80E690E00BD1C4E017D18823CC
:1000A00029F088B38C2788BB76D002D1A895F6CFEB
:1000B00097B1907F97B997B18F70892B87B9369A8E
:1000C000089581E0369980E00895FBDF8823E9F305
:1000D000369824B135B1C901089517B83E9A86B152
:1000E000856086B9379A80E0E3DFEFDF0895EDDFC2
:1000F00096958795969587950895AB9AAA980895B1
:10010000FC0195818AE0989FC00111246FE070E0A6
:10011000F8D066830895CF93E82FF92F40E0CAE026
:100120002FE030E080818C3330F48C9FC0011124AB
:10013000B901E7D060834F5F3196473099F7CF918F
:10014000089581E0B5DFD3DF08951F93CF93DF9348
:10015000D82FC92FF6DF90E08C599F4F6AE070E0EE
:10016000BCD09B01CE01E92FF82F10E0CAE0D0E00F
:10017000408150E0249FC001259F900D349F900D39
:100180001124BE01AAD061931F5F173089F7DF9158
:10019000CF911F910895CF93DF93AB988FE191E0BA
:1001A0000197F1F700C00000C0E6D0E0AA9A95E6FA
:1001B0009A95F1F70000AA9880EC8A95F1F780E013
:1001C00077DF95DF899390E0C736D90779F7AB9A47
:1001D00000000000CE0107979EDFCE01079790DF59
:1001E000CE010797B2DFCE01079795DFCE010797C3
:1001F000DF91CF9108951F920F920FB60F921124A5
:100200008F939F93EF93FF9381B190E0887F883B1A
:100210009105C1F0893B91053CF4883A910559F06C
:10022000803B910581F507C0803C910531F1883C08
:10023000910549F522C081E080936F0080916700AD
:1002400083B915C080916F00863040F010926F0026
:1002500080916D0083B986B78F7B11C0E82FF0E0E5
:10026000E959FF4F908193B98F5F80936F0086B7F4
:10027000806486BF10926E0006C086B7806486BF19
:1002800081E080936E0086B7806886BFFF91EF9112
:100290009F918F910F900FBE0F901F9018958823FC
:1002A00011F481E001C08E7F82B985E486BF089594
:1002B000282F392FD901E7E6F0E08D91819380E076
:1002C000EE36F807D1F710926E00089581E0909114
:1002D0006E00992309F480E00895AA1BBB1B51E12D
:1002E00007C0AA1FBB1FA617B70710F0A61BB70BA6
:1002F000881F991F5A95A9F780959095BC01CD014B
:10030000089597FB092E07260AD077FD04D0E5DF74
:1003100006D000201AF4709561957F4F0895F6F786
:0C032000909581959F4F0895F894FFCFB1
:0E032C00808080808080804242424242424275
:00000001FF
